:1000000000308A002D2A00008A1D0A128A190A1659
:100010008A11831A0F28A500030EA6001428831244
:10002000A500030EA600A6140A08AD00A50E04083C
:10003000A7002008A8002108A9002208AA00230878
:10004000AB002408AC0083128C308400801E2A2868
:100050008C1A4228270884002808A0002908A1003B
:100060002A08A2002B08A3002C08A4002D088A004F
:100070000A1A8A150A12260E83008312250EA61864
:10008000831609008A1184280A108A100A1182072F
:1000900020345434453452344D34253463342034C0
:1000A000303430340A3400344E087F3C0318592869
:1000B00067284E081F3C0318612880304E078400D3
:1000C000642860304E0784004F08800067280034A1
:1000D00051081F3C03187028803051078400732892
:1000E0006030510784000008A10076280034521BBC
:1000F0007E2852080F39A1008328832852080F391F
:10010000093EA100832800348C1E02291A08CC0065
:100110003B1CA8284C08213C031992284C08233C7E
:10012000031DA7280511AE013308B200CE014C080B
:10013000CF0054203B1085144C08233C031DA428F9
:100140000430CD00BB15A7280230CD00BB1101291A
:10015000AE0A2E08803C0319B328BB18B7282F0815
:100160002E02031DB7283B148510051501294C08E4
:100170000D3C0319BF284C080A3C031DE128BB1D98
:10018000DD280130D10068202108CE00D200772080
:10019000210ED000F030D0050230D10068202108B7
:1001A000D100D200772050082104B207B208031D05
:1001B000DB283B15DC288510DE283B153B14051594
:1001C00001292E08CE004C08CF0054204D082E02E5
:1001D000031CF92805304D072E020318F9284D0895
:1001E0002E02363E84004C0800020319F9283B1405
:1001F0000515BB1D01292E08093C031801294C08CF
:10020000B20784288C128A112A28463084000008FC
:1002100003191B290130A100BF30A0006400A00B0E
:100220000E29A10B0C293030A000A00B15290000CD
:100230006400800B0A290034640087140000071052
:100240001C30A000A00B22290000C8014808073C70
:10025000031C37290310C70C031830290710312954
:1002600007141B30A000A00B3329C80A2629000060
:10027000000000000000000007141E30A000A00BCA
:100280003F290000000087100034C61B57290F309B
:10029000A000450EA0050A30200203185229303074
:1002A000A00754294608A0072008C7001C210F30CA
:1002B000C5050A30450203185F2930306129C6138D
:1002C0004608C5074508C7001C218A11F92AA00164
:1002D000A101470803104818A007A00CA10CC818DA
:1002E000A007A00CA10C4819A007A00CA10CC819CC
:1002F000A007A00CA10C481AA007A00CA10CC81ABA
:10030000A007A00CA10C481BA007A00CA10CC81BA7
:10031000A007A00CA10C00342F08D1000B080B057E
:100320008B13A5006820A51B8B1721080F39C5006A
:10033000AF0A2F08D1000B080B058B13A50068200E
:10034000A51B8B172108C60046082F3C0318B729A8
:100350004608393C031CB7294508C7000A30C800C5
:1003600067212108C50046080F39C507AF0A4508AF
:10037000A100BA2900344A08A10149020318C3297F
:100380004908A000CF29A0010830CB00C90DA00D5D
:100390004A0820020318A000A10DCB0BC629003487
:1003A0004818EF29C818072A4708C9006430CA004E
:1003B000BB212008C70021083030031DE42948195B
:1003C000EF29C8192030E6294811C811A1072108D2
:1003D000C9006400490864000C1EEB299900470815
:1003E000C9000A30CA00BB212008C70021083030EC
:1003F000031DFE294819072AC8192030A107210822
:10040000C9006400490864000C1E032A99003030BA
:10041000C7074708C9006400490864000C1E0D2A7C
:10042000990000347B30C9006400490864000C1E48
:10043000162A99004330C9006400490864000C1E64
:100440001E2A99004508C7000130C800D02146087F
:10045000C7000130C800D02100345F30A000213037
:1004600084008001840AA00B312A6030A000A030F3
:1004700084008001840AA00B392AA00184011F3066
:10048000830505308316990022309800903083123E
:10049000980007308316810083121812D03065004F
:1004A000FF306600BC306700871007140E308500EF
:1004B0003230C600052185163B14BB145430B600FB
:1004C0004530B7005230B8004D30B9000608FF3A49
:1004D0000739303EB4003408BA00FB30B3003408AA
:1004E000B30730303402743CB5000A30C1001B3011
:1004F000C2000B138B138B1B7A2A83168C16C03009
:1005000083128B047B30C9006400490864000C1E10
:10051000862A99004130C9006400490864000C1E15
:100520008E2A99000530C60005217B30C900640081
:10053000490864000C1E992A99004D30C9006400D6
:10054000490864000C1EA12A99004630C9006400C5
:10055000490864000C1EA92A9900C31518163B11FE
:10056000BB14AF013B19C52A6400981CBB2A851037
:10057000181200001816431DC42A0B1DC42A0B11A3
:10058000C40BC42A05104311B22A3B112E08BC002B
:10059000BB10BB1DCE2A0A30AF00D02A0830AF00F6
:1005A0002F08AF0AC500D1000B080B058B13A5005F
:1005B0006820A51B8B172108A000513021020319C8
:1005C000EA2A523020020319132B53302002031958
:1005D000232BD42EBB1418123230C6000521243030
:1005E000C7001C21BB1DF92A3508C5003730C600DD
:1005F0004529C50145084420C50AC7001C2105300E
:100600004502031DFA2A3408C7001C210730C60022
:1006100046084420C60AC7001C210B304602031DB1
:10062000082B1816D52E0B138B138B1B142B851030
:10063000051185110830C500FA30C6000521C50B2B
:100640001C2B212BD52E8511AF0A3C082F02031835
:10065000D22E64002F08D1000B080B058B13A500C8
:100660006820A51B8B172108B10031085C3C031DD5
:10067000B42EAF0A2F08D1000B080B058B13A50071
:100680006820A51B8B172108A000623021020319E6
:100690008A2B633020020319A32B65302002031933
:1006A000BC2B663020020319422D6730200203194B
:1006B000582D6830200203195E2D6930200203197D
:1006C000792D6A3020020319942D6B302002031912
:1006D000AE2D6C3020020319C82D6D302002031995
:1006E000E32D6E3020020319FE2D6F302002031916
:1006F0000B2E703020020319242E723020020319B1
:100700003D2E743020020319432E78302002031945
:10071000542EB22E7B30C9006400490864000C1EC0
:100720008E2B99004230C9006400490864000C1EF9
:10073000962B99004530C9006400490864000C1EDE
:100740009E2B9900B32E7B30C900640049086400D9
:100750000C1EA72B99004230C900640049086400B0
:100760000C1EAF2B99004430C90064004908640096
:100770000C1EB72B9900B32E0230AF07B1012F0822
:10078000D1000B080B058B13A5006820A51B8B1748
:100790002108B00030082F3C0318E72B3008393C03
:1007A000031CE72B8C212108B0002F08D1000B0877
:1007B0000B058B13A5006820A51B8B1721083B3C5C
:1007C000031DE62BAF0A8C212108B100E82BB001F4
:1007D000C3102F08D1000B080B058B13A500682050
:1007E000A51B8B172108A0004130210203193D2CC5
:1007F000423020020319462C4330200203194F2CAB
:10080000443020020319582C483020020319612C6F
:10081000663020020319662C6730200203196B2C06
:100820006A30200203197C2C4B3020020319812CE2
:100830004A3020020319902C4D3020020319AB2CB2
:100840004E3020020319C82C4F3020020319E52C2A
:10085000503020020319022D7330200203191F2D7E
:10086000753020020319252D6830200203192A2D26
:100870006C3020020319312D382D3E083002031848
:10088000442C3008BE02452CBE013A2D3008BE076C
:100890003E08410203184E2C4108BE003A2D300894
:1008A000BD073D0842020318572C4208BD003A2DEF
:1008B0003D08300203185F2C3008BD02602CBD01DA
:1008C0003A2D3008BE003108BD003A2D3008BE0078
:1008D0003108BD003A2D30080A3C0318712C0A304B
:1008E000B00005143008C7000A30C800672121088D
:1008F000C400810143153A2D3008BE003108BD0007
:100900003A2D3D08B00030084202031C8F2C6400D1
:10091000203064000C1E892C9900B00A832C3A2DDB
:100920003008023C031DA92C7B30C9006400490833
:1009300064000C1E982C99004130C90064004908DD
:1009400064000C1EA02C99000530C6000521BD01D5
:10095000BE01C3143A2DC31DC62C3008073C031C2E
:10096000C62C7B30C9006400490864000C1EB52CFD
:1009700099004630C9006400490864000C1EBD2C73
:1009800099003008C7000C30C800D021C3143A2D9C
:10099000C31DE32C3008073C031CE32C7B30C9004B
:1009A0006400490864000C1ED22C99004530C9002F
:1009B0006400490864000C1EDA2C99003008C70056
:1009C0000C30C800D021C3143A2DC31D002D3008AF
:1009D000073C031C002D7B30C900640049086400FB
:1009E0000C1EEF2C99004430C900640049086400D3
:1009F0000C1EF72C99003008C7000C30C800D0211D
:100A0000C3143A2DC31D1D2D3008073C031C1D2D9A
:100A10007B30C9006400490864000C1E0C2D99004D
:100A20004930C9006400490864000C1E142D990067
:100A30003008C7000C30C800D021C3143A2D3D083F
:100A4000BF003E08C000C3143A2D3F08BD00400857
:100A5000BE003A2D3008073C031D2F2D4314C3144C
:100A60003A2D3008073C031D362D4310C3143A2D90
:100A7000C3143A2DC318412D3D08C5003E08C600D9
:100A80001222B32E7B30C9006400490864000C1E9A
:100A9000462D99004130C9006400490864000C1ECD
:100AA0004E2D99000530C6000521BD01BE01B32EB3
:100AB00005140630C40081014315B32EC31D782DE3
:100AC0007B30C9006400490864000C1E642D990045
:100AD0004B30C9006400490864000C1E6C2D99005D
:100AE0004530C9006400490864000C1E742D99004B
:100AF000B32EC31D932D7B30C900640049086400E8
:100B00000C1E7F2D99004B30C90064004908640019
:100B10000C1E872D99004430C90064004908640008
:100B20000C1E8F2D9900B32E7B30C900640049083C
:100B300064000C1E982D99004D30C90064004908CE
:100B400064000C1EA02D99004630C90064004908BD
:100B500064000C1EA82D9900C315B32E7B30C9006C
:100B60006400490864000C1EB22D99004D30C90084
:100B70006400490864000C1EBA2D99004D30C9006C
:100B80006400490864000C1EC22D9900C311B32EE5
:100B9000C31DE22D7B30C9006400490864000C1EAF
:100BA000CE2D99004A30C9006400490864000C1E2B
:100BB000D62D99004430C9006400490864000C1E19
:100BC000DE2D9900B32EC31DFD2D7B30C9006400BE
:100BD000490864000C1EE92D99004A30C9006400E0
:100BE000490864000C1EF12D99004530C9006400CD
:100BF000490864000C1EF92D9900B32EBD0141086F
:100C00003E02031D052EBE01062EBE0AC5013E088A
:100C1000C6001222B32E7B30C9006400490864006C
:100C20000C1E0F2E99004730C9006400490864006B
:100C30000C1E172E99004530C90064004908640055
:100C40000C1E1F2E9900B32E7B30C900640049088A
:100C500064000C1E282E99004730C9006400490822
:100C600064000C1E302E99004430C900640049080D
:100C700064000C1E382E9900B32EBD01C5013E083C
:100C8000C6001222B32E01303D070339043CBD07D4
:100C90003D08420203184E2E4208BD003D08C50023
:100CA0003E08C6001222B32EAF0A2F08D1000B084F
:100CB0000B058B13A5006820A51B8B172108C50009
:100CC000D2000B080B058B13A5007720A51B8B17F3
:100CD000210EC700F030C705AF0A2F08D1000B085E
:100CE0000B058B13A5006820A51B8B172108C800D6
:100CF000D2000B080B058B13A5007720A51B8B17C3
:100D000047082104B1007B30C90064004908640031
:100D10000C1E872E99005430C900640049086400F5
:100D20000C1E8F2E9900310864000C1E942E990021
:100D30001B3064000C1E992E9900BD0A3D0842022A
:100D40000318B12EBD014318AC2E41083E02031D0D
:100D5000AB2EBE01AC2EBE0A3D08C5003E08C60043
:100D60001222B32EB32ED12E31087B3C0319D12E83
:100D7000310864000C1EB92E9900BD0A3D084202DC
:100D80000318D12EBD014318CC2E41083E02031D8D
:100D9000CB2EBE01CC2EBE0A3D08C5003E08C600C3
:0E0DA0001222242B8515D52ED52EB02A6300E5
:02400E00C500EB
:00000001FF
